:1000000000308A003C2A00000030A1001F08C339DC
:1000100021049F000D30A000A00B0C289F149F18F6
:100020000F281E08A601A500260CA300250CA2007F
:10003000A30CA20CA30CA20CA30CA20C2208AD00D2
:10004000A50DA60DA50DA60DFC30A5050430A1003B
:100050001F08C33921049F000D30A000A00B2E28DB
:100060009F149F1831281E08A801A700280CA30080
:10007000270CA200A30CA20CA30CA20CA30CA20C94
:100080002208AE00270DAB00280DAC00AB0DAC0D67
:10009000FC30AB050C30A1001F08C33921049F00C0
:1000A0000D30A000A00B52289F149F1855281E0841
:1000B000AA01A90000344F308400000803196D28FC
:1000C0000230A100A001A00B6328A10B6228973089
:1000D000A000A00B6928800B60280034CF014F08D6
:1000E000293C031C822805150830A000A00B7628A7
:1000F000000005110330A000A00B7C2800000000C8
:10010000CF0A6F280034CF014F08143C031C9728F6
:1001100005150830A000A00B8B2800000511033046
:10012000A000A00B912800000000CF0A8428003412
:100130000830D002031CA728503084000310800C24
:1001400000080319A728A5280000800BA428003464
:10015000AA08031DB0282908DB3C031CB02885161B
:1001600000340130B800B901BA01BB00BC00CC01B9
:10017000042005118512310BC028BD01BE01C6281F
:10018000B108031DC628BD010130BE002D080F3C7B
:10019000031DCC280E30AD00CE014E08033C031CDD
:1001A000E9280F30AD052D08B4000130B405340B3B
:1001B000E0284E080A3C383E840001308000E528E3
:1001C0004E080A3C383E840080010310AD0CCE0A74
:1001D000CD28851DF8280B30CE004E080E3C031CA0
:1001E000F72838304E0784008001CE0AED281E29FA
:1001F0002E08053C031C0B290B30CE004E080E3C8C
:10020000031C0A2938304E0784000130800085160F
:10021000CE0AFE281E292E08093C03181E290B3081
:10022000CE004E080D3C031C1C2938304E078400BC
:1002300080018516CE0A11290130C6002E08063C21
:10024000031C3C290130C7002E08023C031C2C294A
:10025000C8010130C9003B292E08043C031C342985
:100260000130C800C9013B292E08063C031C3B296C
:100270000130C800C9005729C7012E08083C031CDB
:100280004429C801C90157292E080A3C031C4C29DE
:10029000C8010130C90057292E080C3C031C542901
:1002A0000130C800C90157290130C800C900B30195
:1002B0000330CE004E080F3C031C6D2938304E072A
:1002C00084000310000DB30701304E07383E840050
:1002D0000008B3070230CE075A29490B72290310D0
:1002E000490DB3070330B305B308031D7B29013063
:1002F000CA00CB008F29330B8129CA010130CB0002
:100300008F293308023C031D89290130CA00CB0123
:100310008F293308033C031D8F29CA01CB016E20AE
:1003200083200130CE004E08143C031CAF29383026
:100330004E078400000BA5296E200330CF00C63085
:10034000D0009820CF0B9F29AD2983200330CF0008
:10035000C630D0009820CF0BA829CE0A93290511CA
:10036000A820C830CF005B20982AA101A201A001DB
:10037000A3015608031DBF2955080319D9291030B8
:10038000D7000310D30DD40DA00DA30D56082302E2
:10039000031DCC2955082002031CD5295508A002AD
:1003A000031CA3035608A3020314A10DA20DD70B2F
:1003B000C1290000032AD201D101D208031DF52969
:1003C0005108123C031CF52905150830A000A00BAC
:1003D000E729000005110330A000A00BED29000063
:1003E0000000D10A0319D20ADD290511D830A00076
:1003F000A00BF82900004F08D4004E08D300D60106
:100400000A30D500B5292208CF002108CE00D2013C
:10041000D10152084F02031C1D2A031D132A4E0846
:10042000510203181D2A0130D00000000000000016
:100430000000D10A0319D20A092A00340420051148
:1004400085122C08CF002B08CE00DB210230CF0014
:10045000CE01DB212608CF002508CE00DB210230AB
:10046000CF00CE01DB210230CF00CE01DB21A8205E
:100470000A30CF005B209C2A84011F3083051F13A4
:1004800083161F149F141F159F15073083129F009A
:10049000703083168F001B30650083121F13831684
:1004A0001F149F141F119F151F129F161F138312D5
:1004B0009F131F14703083168F008312851204203F
:1004C000851D662A0130B600B701692AB6010130E0
:1004D000B7002D080C3C0318712AB1010330B2009B
:1004E000752A0130B1000230B2002D08043C031817
:1004F0007B2A0420752ACD0132084D0203188A2A6E
:100500008516FA30CF005B208512FA30CF005B20D1
:10051000CD0A7C2A370B952A85160230CE00FA3098
:10052000CF005B20CE0B8F2A8512360B992AB1287B
:0C053000952A370B9D2A1E2A992A630089
:02400E00C43FAD
:00000001FF
